:1000000019C049CB189518951895189518951895F5
:100010001895189518951895189518951895189578
:100020001895189518951895189518951895189568
:10003000189518958FEF8DBFC0ECE8E54E2E84E043
:100040008EBFD4E0F4E05F2E662486E880937A00C9
:1000500080E480937C0052985398E894ABE2B0E03F
:100060008C9182F98C93E894ABE2B0E08C9183F9A7
:100070008C93FBD680916900836080936900E89A35
:1000800078948FE384B988E385B980E087B98EEFEF
:1000900088B980E08AB983EF8BB980E080934B0107
:1000A00080E090E0A0E5B1E08D939C9380E090E04B
:1000B000A2E5B1E08D939C93ADE4B1E0BA93AA932D
:1000C000AFD82296F8D827D95A924A928FE0A42D19
:1000D000B52D8C9381E0AFDAD8D8229681E0A7DAEB
:1000E0005A924A9288E5A42DB52D8C9381E0A3DA2B
:1000F000C8D7229681E09BDA88E580933E0180E0B4
:1001000090E0A6E4B1E08D939C93A9E2B0E00C915D
:1001100003FB00270EF401E040E0041709F00EC0D5
:10012000A6E4B1E08CDAA6E4B1E00D911C91083EA2
:1001300053E0150709F001C098D6E7CFA2E3B1E07C
:100140000C9107FB00270EF401E041E0041709F0D1
:100150001DC0A2E3B1E00C9104FB00270EF401E006
:1001600041E0041709F006C0A8E1B1E0BA93AA93F0
:1001700087D422966894A2E3B1E08C9186F98C939F
:10018000E894A2E3B1E08C9187F98C930027A9E26F
:10019000B0E08C9181FB0EF401E040E0041781E0B7
:1001A00009F080E08F9300913E010F3F81E009F458
:1001B00080E09F918923882309F40FC08FEF8093FB
:1001C0003E015A924A928FEFA42DB52D8C9381E077
:1001D00032DA64D6229681E02ADA0027A9E2B0E07A
:1001E0008C9181FB0EF401E041E0041781E009F0FD
:1001F00080E08F9300913E010F3F81E009F080E0A5
:100200009F918923882309F40FC088E580933E01DC
:100210005A924A9288E5A42DB52D8C9381E00BDA91
:100220003DD6229681E003DAE2EFF5E1A8E4B1E001
:100230008C919927A8E3B1E0D8DBE2E0F6E1A8E4ED
:10024000B1E08C919927A9E3B1E0CFDB00913701B0
:10025000003081E009F080E08F9300913E01063488
:1002600081E009F080E09F91892B8F9300913E01FE
:100270000F3F81E009F080E09F91892B882309F4EA
:1002800033C08FE090E0A9E4B1E08D939C93A9E4A2
:10029000B1E08D919C91A2E4B1E08D939C9395E0A7
:1002A000A9E4B1E07CDBA2E4B1E00D911C91A9E4EA
:1002B000B1E04D915C91042B152BA2E4B1E00D93BC
:1002C0001C9395E0A9E4B1E06ADBA2E4B1E00D91F2
:1002D0001C91A9E4B1E04D915C91042B152BA2E493
:1002E000B1E00D931C9352C180E090E0A2E4B1E034
:1002F0008D939C9300913E01083581E009F080E0E8
:100300008F9300913E01093581E009F080E09F91D3
:10031000892B882309F4ABC00027A6E2B0E08C91BA
:1003200084FB0EF401E040E0041709F009C0A8E3E3
:10033000B1E08C91A2E4B1E08D9388278C931AC030
:100340000027A6E2B0E08C9182FB0EF401E040E0D1
:10035000041709F009C0A9E3B1E08C91A2E4B1E06F
:100360008D9388278C9306C08FE090E0A2E4B1E0E3
:100370008D939C930027A6E2B0E08C9183FB0EF452
:1003800001E040E0041709F01BC0A8E3B1E08C9144
:10039000A9E4B1E08D9388278C9395E0A9E4B1E0BE
:1003A000FEDAA2E4B1E00D911C91A9E4B1E04D9117
:1003B0005C91042B152BA2E4B1E00D931C933EC07D
:1003C0000027A6E2B0E08C9185FB0EF401E040E04E
:1003D000041709F01BC0A9E3B1E08C91A9E4B1E0D6
:1003E0008D9388278C9395E0A9E4B1E0D8DAA2E454
:1003F000B1E00D911C91A9E4B1E04D915C91042B09
:10040000152BA2E4B1E00D931C9318C08FE090E08F
:10041000A9E4B1E08D939C9395E0A9E4B1E0BFDA43
:10042000A2E4B1E00D911C91A9E4B1E04D915C9181
:10043000042B152BA2E4B1E00D931C938FE090E008
:10044000A9E4B1E08D939C939AE0A9E4B1E0A7DA26
:10045000A2E4B1E00D911C91A9E4B1E04D915C9151
:10046000042B152BA2E4B1E00D931C938FC00091D7
:100470003E010A3509F08AC00027A6E2B0E08C915F
:1004800083FB0EF401E040E0041709F01BC0A8E371
:10049000B1E08C91A9E4B1E08D9388278C939AE028
:1004A000A9E4B1E07CDAA2E4B1E00D911C91A9E4E9
:1004B000B1E04D915C91042B152BA2E4B1E00D93BA
:1004C0001C933EC00027A6E2B0E08C9185FB0EF4A1
:1004D00001E040E0041709F01BC0A9E3B1E08C91F2
:1004E000A9E4B1E08D9388278C939AE0A9E4B1E068
:1004F00056DAA2E4B1E00D911C91A9E4B1E04D916E
:100500005C91042B152BA2E4B1E00D931C9318C051
:100510008FE090E0A9E4B1E08D939C939AE0A9E488
:10052000B1E03DDAA2E4B1E00D911C91A9E4B1E0A3
:100530004D915C91042B152BA2E4B1E00D931C931B
:100540008FE090E0A9E4B1E08D939C93A2E4B1E048
:100550000D911C91A9E4B1E04D915C91042B152BF8
:10056000A2E4B1E00D931C9395E0A9E4B1E017DAA1
:10057000A2E4B1E00D911C91A9E4B1E04D915C9130
:10058000042B152BA2E4B1E00D931C9322D780E03D
:1005900090E0AAE3B1E08D939C93A9E2B0E08C9146
:1005A00081FB882780F9809580FBAAE3B1E08C91DC
:1005B00084F98C9300913E01083509F03AC000910E
:1005C0004B01013009F007C06894AAE3B1E08C91B7
:1005D00081F98C930BC000914B01023009F006C0E9
:1005E0006894AAE3B1E08C9180F98C930027A9E28A
:1005F000B0E08C9184FB0EF401E040E0041709F0B8
:1006000006C06894AAE3B1E08C9185F98C93002729
:10061000A9E2B0E08C9180FB0EF401E040E0041709
:1006200009F006C06894ABE3B1E08C9186F98C9335
:10063000E0C000913E01093509F03AC000914B013C
:10064000013009F007C06894AAE3B1E08C9182F907
:100650008C930BC000914B01023009F006C06894E6
:10066000AAE3B1E08C9183F98C930027A9E2B0E072
:100670008C9184FB0EF401E040E0041709F006C001
:100680006894AAE3B1E08C9186F98C930027A9E2E3
:10069000B0E08C9180FB0EF401E040E0041709F01B
:1006A00006C06894ABE3B1E08C9186F98C93A1C04D
:1006B00000913E010A3509F03AC000914B0101302A
:1006C00009F007C06894ABE3B1E08C9180F98C939A
:1006D0000BC000914B01023009F006C06894ABE3F7
:1006E000B1E08C9181F98C930027A9E2B0E08C9164
:1006F00084FB0EF401E040E0041709F006C06894A2
:10070000AAE3B1E08C9187F98C930027A9E2B0E0CD
:100710008C9180FB0EF401E040E0041709F006C064
:100720006894ABE3B1E08C9186F98C9362C0009140
:100730003E01063409F05DC000914B01013009F023
:1007400007C06894ABE3B1E08C9182F98C930BC045
:1007500000914B01023009F006C06894ABE3B1E0B0
:100760008C9183F98C930027A9E2B0E08C9184FBF3
:100770000EF401E040E0041709F006C06894ABE312
:10078000B1E08C9184F98C930027A6E2B0E08C91C3
:1007900084FB0EF401E040E0041709F006C0689401
:1007A000ABE3B1E08C9185F98C930027A6E2B0E031
:1007B0008C9182FB0EF401E040E0041781E009F027
:1007C00080E08F930027A9E2B0E08C9180FB0EF4CB
:1007D00001E040E0041781E009F080E09F91892367
:1007E000882309F406C06894ABE3B1E08C9187F9E3
:1007F0008C93A4E4B1E04D915C91A2E4B1E00D9141
:100800001C910417150781E009F480E08F93ACE395
:10081000B1E04D915C91AAE3B1E00D911C910417F8
:10082000150781E009F480E09F91892B8F93009157
:100830004101003081E009F080E09F91892B8823FD
:1008400009F43DC0A4E2B1E00C9105FB00270EF4D1
:1008500001E041E0041709F032C0A2E4B1E08D915B
:100860009C91A4E4B1E08D939C93A2E4B1E08C91BF
:10087000A6E2B1E08C93A2E4B1E011968C91A7E2DC
:10088000B1E08C93AAE3B1E08C91A8E2B1E08C9343
:10089000AAE3B1E011968C91A9E2B1E08C93A4E2B5
:1008A000B1E0BA93AA935A924A9284E0A42DB52D4E
:1008B0008C9381E0C0D656D2249681E0B8D600272A
:1008C000A5E3B1E08C9187FB0EF401E041E0041751
:1008D00009F011C00027A6E2B0E08C9181FB0EF474
:1008E00001E041E0041709F005C0809135018F77E0
:1008F0008093350162C00027A6E2B0E08C9181FBB5
:100900000EF401E040E0041781E009F080E08F93ED
:1009100000913E010F3F81E009F480E09F9189231F
:100920008F93A0E1B0E0BA93AA9307D42296003047
:1009300081E009F080E09F918923882309F43DC07C
:100940008091350180688093350100913E010A3520
:1009500009F00DC05A924A9286E4A42DB52D8C93CD
:1009600081E069D69BD2229681E061D626C00091B3
:100970003E01063409F00DC05A924A9288E5A42D32
:10098000B52D8C9381E057D689D2229681E04FD63F
:1009900014C000913E0141E0040FA6E3B1E00C93C6
:1009A0005A924A9280913601A42DB52D8C9381E004
:1009B00042D674D2229681E03AD6C4D5A0CBF89420
:1009C000FFCF121201100100000008AAAA02EF01D5
:1009D00000010200010022090222000101028096AA
:1009E0000904000001030000000921110100012297
:1009F00040000705810308000A004105010905A11F
:100A0000010901A1000933093409351500251E9596
:100A100003750581029501750181030930093115BE
:100A2000FF2501950275028102C005091901290CF3
:100A300015002501950C75018102C000040403090D
:100A400004000E0E0363006E0063006A006F0079FD
:100A500000002C2C0369006B00610072006900200B
:100A60000063006E00630020006A006F007900736D
:100A7000007400690063006B002000760031000004
:100A800080E08093340180E6A881B9818C93009145
:100A90000201003809F03EC000910301063009F060
:100AA00038C000910501013009F007C0E2ECF9E01F
:100AB000B0D581E0809334012CC0023009F007C02A
:100AC000E6EDF9E0A6D581E08093340122C0033041
:100AD00009F01FC000910401003009F007C0ECE3E9
:100AE000FAE097D581E08093340113C0013009F01A
:100AF00007C0E2E4FAE08DD581E08093340109C0BB
:100B0000023009F006C0E2E5FAE083D581E0809387
:100B100034016CC0003009F03AC000910301053087
:100B200009F021C0A881B981BA93AA935A924A9236
:100B300080E0A42DB52D8C9381E07DD513D1249632
:100B400081E075D5A881B9810C9105FB00270EF4D1
:100B500001E040E0041709F001C0F4CF80910401E6
:100B60008093000113C0093009F010C0A881B98139
:100B7000BA93AA935A924A9280E0A42DB52D8C93F1
:100B800081E059D5EFD0249681E051D52FC00138AE
:100B900009F011C000910301063009F00BC000916B
:100BA0000501023209F006C0EAEFF9E032D581E032
:100BB000809334011BC0013209F018C00091030179
:100BC0000A3009F013C081E080934101A881B98106
:100BD000BA93AA935A924A9280E0A42DB52D8C9391
:100BE00081E029D5BFD0249681E021D50091340140
:100BF000013009F00AC0A881B981BA93AA93A8E08C
:100C0000B1E0BA93AA9302D02496089581E03DD52D
:100C100081E03BD581E039D582E037D5FDD4AE8186
:100C2000BF81D3D60C92F5D4AE81BF814C91A885FB
:100C3000B9850C91041708F006C0A885B9858C9178
:100C4000AE81BF818C9382E0AC81BD818C9381E0C9
:100C5000AA81BB818C93AE81BF814C91AA81BB815B
:100C60000C91041710F009F077C0AC81BD818C9114
:100C70008F5F8C93D1D4AC81BD81AD90BB24AA850C
:100C8000BB85AA0DBB1D1197A0D60C92C2D4AC8116
:100C9000BD810C910A3081E009F080E08F93AE8134
:100CA000BF814C91AA81BB810C91041781E009F0AE
:100CB00080E09F91892B882309F447C0AC81BD81D6
:100CC0008C9182508C93AA85BB85BA93AA935A9231
:100CD0004A92A885B9858C91A42DB52D8C9381E07D
:100CE000AAD440D0249681E0A2D4AA85BB850C91D9
:100CF00005FB00270EF401E040E0041709F021C0D5
:100D000080E090E0A881B9818D939C93A9E2B0E046
:100D10000C9103FB00270EF401E040E0041709F0FA
:100D20000FC0A881B9818BD4A881B9810D911C9184
:100D3000083E53E0150709F002C097D00DC0E6CF7A
:100D4000D4CF82E0AC81BD818C93AA81BB818C9190
:100D50008F5F8C9308F47FCF85E0481A8827580A64
:100D600028960895AA81BB818C91807C8C9380E029
:100D700090E0A0E3B1E08D939C93A881B9810C91A0
:100D8000003009F41BC081E08A9381E08A93AA8134
:100D9000BB818C918A934FEF5FEF25E030E8AD8007
:100DA000BE80A2E0B0E0AA0DBB1D22D6A0E3B1E058
:100DB0004D935C93A0E3B1E042E031D4A881B981C6
:100DC0008C918D5F8C93AA81BB810C91A881B98194
:100DD0004C91040FAA81BB810C93A0E3B1E08C91EC
:100DE000A881B981AD90BB24AA81BB81AA0DBB1D8E
:100DF00011978C93A881B9818C918F5F8C93A0E31C
:100E0000B1E011968C91A881B981AD90BB24AA81E3
:100E1000BB81AA0DBB1D11978C938BE4AA80BB806C
:100E2000A1E0B0E0AA0DBB1D8C93AA81BB810C91FF
:100E300006FB00270EF401E040E0041709F008C0AB
:100E400083ECAA80BB80A1E0B0E0AA0DBB1D8C930F
:100E50006894AA81BB818C9184F98C93E894AA81CF
:100E6000BB818C9185F98C9308956894A2E3B1E0DD
:100E70008C9186F98C93E894A2E3B1E08C9187F988
:100E80008C9380E28093180180E28093240180E0BB
:100E90008093000180E080934101089587E090E015
:100EA000A4E5B1E08D939C9380E08093570100917D
:100EB0005701083010F009F0DEC080E08093360161
:100EC00000913601073010F009F0C8C000913601DA
:100ED00041E0040FAFE3B1E00C93A4E5B1E04D9124
:100EE0005C91A6E3B1E00D9111270417150714F0EA
:100EF00009F001C051C00091360140915401041B1A
:100F0000A6E5B1E00C938091560181508093560183
:100F1000A881B9810C91063409F00AC0EAECF5E128
:100F2000A6E5B1E08C919927A0E4B1E05ED533C08D
:100F3000083509F00AC0E2EDF5E1A6E5B1E08C91D3
:100F40009927A0E4B1E051D526C0093509F00AC0BF
:100F5000EAEDF5E1A6E5B1E08C919927A0E4B1E0D6
:100F600044D519C00A3509F00AC0E2EEF5E1A6E55C
:100F7000B1E08C919927A0E4B1E037D50CC00F3FC8
:100F800009F009C0EAEEF5E1A6E5B1E08C919927F8
:100F9000A0E4B1E02AD55AC0A4E5B1E04D915C913E
:100FA000A6E3B1E00D9111270417150709F004C05D
:100FB00080E0809340014AC0009136014091570182
:100FC000040FA6E5B1E00C9300913E01063409F050
:100FD0000AC0EAECF5E1A6E5B1E08C919927A0E41E
:100FE000B1E003D533C0083509F00AC0E2EDF5E100
:100FF000A6E5B1E08C919927A0E4B1E0F6D426C033
:10100000093509F00AC0EAEDF5E1A6E5B1E08C91F9
:101010009927A0E4B1E0E9D419C00A3509F00AC063
:10102000E2EEF5E1A6E5B1E08C919927A0E4B1E00C
:10103000DCD40CC00F3F09F009C0EAEEF5E1A6E5EB
:10104000B1E08C919927A0E4B1E0CFD47DD1A6E3A3
:10105000B1E08C918F5F8C9308F432CFA4E5B1E0BE
:10106000F5D28EE190E002D3A7E5B1E08C918F5FDD
:101070008C9308F41CCFA881B9818C9180933E0198
:10108000089580E08093360100913601073010F01A
:1010900009F052C00091360141E0040FAFE3B1E026
:1010A0000C93A881B9810C91063409F00AC0EAECCE
:1010B000F5E1A6E3B1E08C919927A0E4B1E095D4E5
:1010C00033C0083509F00AC0E2EDF5E1A6E3B1E06E
:1010D0008C919927A0E4B1E088D426C0093509F0A5
:1010E0000AC0EAEDF5E1A6E3B1E08C919927A0E40E
:1010F000B1E07BD419C00A3509F00AC0E2EEF5E18F
:10110000A6E3B1E08C919927A0E4B1E06ED40CC0C5
:101110000F3F09F009C0EAEEF5E1A6E3B1E08C91DA
:101120009927A0E4B1E061D40FD1A6E3B1E08C919E
:101130008F5F8C9308F4A8CF08950027A9E2B0E050
:101140008C9184FB0EF401E040E0041781E009F08B
:1011500080E08F930027A9E2B0E08C9181FB0EF430
:1011600001E040E0041781E009F080E09F91892BC5
:101170008F930027A9E2B0E08C9180FB0EF401E090
:1011800040E0041781E009F080E09F91892B8F9364
:101190000027A6E2B0E08C9185FB0EF401E040E070
:1011A000041781E009F080E09F91892B8F9300273D
:1011B000A6E2B0E08C9183FB0EF401E040E004175E
:1011C00081E009F080E09F91892B8F930027A6E2B0
:1011D000B0E08C9184FB0EF401E040E0041781E064
:1011E00009F080E09F91892B8F930027A6E2B0E061
:1011F0008C9182FB0EF401E040E0041781E009F0DD
:1012000080E09F91892B882309F405C081E0A881A3
:10121000B9818C9304C080E0A881B9818C93089532
:101220000027A9E2B0E08C9187FB0EF401E040E0DA
:10123000041709F005C081E0A881B9818C9324C00E
:101240000027A9E2B0E08C9186FB0EF401E040E0BB
:10125000041709F005C082E0A881B9818C9314C0FD
:101260000027A9E2B0E08C9185FB0EF401E040E09C
:10127000041709F005C083E0A881B9818C9304C0EC
:1012800080E0A881B9818C930895A881B9810C91DF
:101290000F3010F009F001C004C08FE0A881B981BF
:1012A0008C938AE080933F01A881B9818C918093CF
:1012B00040014AD008958CE080933F0180E0809304
:1012C000400142D089E080933F0180E0809340015B
:1012D0003BD05A924A9287E0A42DB52D8C9381E0A1
:1012E000AAD1D3DF229681E0A2D18BE080933F0187
:1012F00087E08093400128D08FE080933F0180E019
:101300008093400121D08CE080933F0181E0809365
:1013100040011AD0089581E0809336010091360192
:10132000083010F009F00FC08091360180933F0122
:1013300080E08093400108D0A6E3B1E08C918F5FFC
:101340008C9308F4EBCF0895F89429982A9828985C
:10135000219A229A2A98AFE3B1E0119698E08E91F3
:10136000983018F4392F992702C038E09850881F18
:10137000299808F4299A000000002A9A0000000029
:101380002A98000000003A9591F7992341F7219A95
:10139000229A2A98A0E4B1E0119698E08E919830B4
:1013A00018F4392F992702C038E09850881F2998DF
:1013B00008F4299A000000002A9A000000002A98E8
:1013C000000000003A9591F7992341F7289A789404
:1013D0000895ACE4B1E0BA93AA9322DF229640913B
:1013E0004D0100914C01041781E009F480E08F93D6
:1013F00000914C01003081E009F480E09F91892345
:10140000882309F433C0ACE4B1E00D911127ADE4B9
:10141000B1E04D915527041B150BAEE4B1E00D93DF
:101420001C93AEE4B1E00D911C91013050E0150722
:1014300081E009F080E08F93AEE4B1E00D911C9162
:101440000E3F5FEF150781E009F080E09F91892B47
:10145000882309F404C0A0E5B1E0F8D003C0A0E5FA
:10146000B1E0EDD080914C0180934D0100914B0192
:10147000003009F02FC0A0E5B1E00D911C910030C3
:1014800050E015070CF401C00DC081E080934B01C2
:1014900080E496E0A2E5B1E08D939C93A0E5B1E0F5
:1014A000CED017C0A0E5B1E00D911C91003050E006
:1014B000150714F009F001C00CC082E080934B01C5
:1014C00080E496E0A2E5B1E08D939C93A0E5B1E0C5
:1014D000BDD037C0A2E5B1E00D911C91003050E0C5
:1014E000150714F009F001C02CC0A2E5B1E0AED0A0
:1014F000A2E5B1E00D911C91003050E0150714F009
:1015000009F01FC000914B01013081E009F080E03B
:101510008F9300914B01023081E009F080E09F91B0
:10152000892B882309F40AC082E390E0A2E5B1E0A8
:101530008D939C9383E080934B0103C080E0809364
:101540004B01089500917C00007F006000937C00B7
:101550000FD2A9E4B1E08D939C9396E0A9E4B1E0A9
:1015600029D2809149018093480191E0A9E4B1E03A
:1015700021D2A9E4B1E04D915C91A7E3B1E00D91D6
:1015800011270417150709F41FC0809149018093A2
:101590003701A7E3B1E08C9180FBA5E2B0E08C912C
:1015A00085F98C93A7E3B1E08C9181FBA5E2B0E0D3
:1015B0008C9184F98C93A7E3B1E08C9182FBA5E236
:1015C000B0E08C9183F98C9308950303031F1F03EC
:1015D0007F7F00C3663C183C66C300181818183C8F
:1015E00066E700FFFE0C18307FFF7F7F77777F2252
:1015F000221C0F0F0909080807070605040302014A
:1016000000000F0F15151616171718191A1B1C1D99
:101610001E1E8E2E9F2E0895E82DF92D0895EA2F77
:10162000FB2F8D91809581934A95D9F70895481A9B
:101630008827580A0895480E8827581E0895ED9166
:10164000FC91EF5FFF4FFC93EE930895ED91FC91B9
:10165000E150F040FC93EE9308953197F1F708952F
:10166000689462F80895E89462F80895EF93FF9300
:10167000EE27E82BE92B31F0E8EBFBE03197F1F7AF
:101680000197D1F7FF91EF9108955A924A92480E2F
:101690008827581E0895AF93BF934F930F931F93BE
:1016A0002F933F933FB73F9333954B9BE9F74A996D
:1016B00007C04B9B05C04A9903C04B9B01C07EC02D
:1016C000A1E0B1E030913201442736FF4BE0A40F96
:1016D00040E0B41F4B99EBCF2FE704E03FEF00C091
:1016E000000019B100C004C019B132273D933FEF8B
:1016F000012702FB20F909B1297FA1F10C7089F1C2
:10170000102712FB21F919B10000237F89F1000095
:10171000012702FB22F909B1277E81F1102712FB74
:1017200023F92F7C89F119B1012702FB24F900C0AC
:101730002F7979F109B12F774395102712FB25F9FD
:101740002F7361F119B1012702FB26F9223058F1FC
:101750004C30A0F509B1102712FB27F9243040F1D5
:10176000C3CF39C021603E7F1095000009B1C6CFBC
:1017700022603D7F009519B10000C9CF2B7F3460F6
:101780001095000009B1CACF2860377F009500C0CE
:10179000CACF20613F7E109500C0CCCF20623F7D34
:1017A000009500C0CFCF20643F7B109500C0D2CF02
:1017B00020683F77009500C000C096CF3CB330FD55
:1017C00073CF3F913FBF3F912F911F910F914F9149
:1017D000BF91AF91189531E03CBBA41BB0400D9177
:1017E000102F13731132C1F41D912D9140910001FE
:1017F000110F221F16952F70141751F5093649F055
:10180000013E41F13091320136FF22C00D3209F123
:101810001FC02093330149F02091330125FDCECF25
:1018200030913201307C322B2F70A8E1B1E02030B2
:1018300029F0A4E2B1E0213009F00AC01D91093677
:1018400091F0033CB9F00B34A9F0023D31F0B6CF72
:101850002062206120933301B1CF1F7E106230E4FB
:1018600013271E93ABCF14FF03C0412F4F7022C02C
:101870001AE50BC0433041F036FFFACF30683F7BAA
:10188000309332014093170112EDBB27A1E141E0F3
:1018900011C05BB9279520F43A9521F4220FF9CFB6
:1018A000502736E000C05BB92795B8F43A95B9F4F3
:1018B000220FF9CF5F934F930CE05B9A2AB12C6013
:1018C0002AB95BB120E4502736E000005BB92795C8
:1018D00078F43A9579F4220FF9CF502736E02D911C
:1018E0005BB927958EF178F73A9579F7220FF9CF02
:1018F000502736E000C05BB9279520F43A9521F4D3
:10190000220FF9CF502736E000C05BB9279520F4AD
:101910003A9521F4220FF9CF502736E000C05BB989
:10192000279520F43A9521F4220FF9CF502736E07D
:101930004A9547FB5BB9279520F43A9521F4220F8D
:10194000F9CF502736E0A5CF00C02BB1237F2BB9AC
:101950004F91A41BB040422F28603AB1337F01E081
:101960000CBB5F910E9103742BB93AB94BB926CFDA
:1019700070917A00706470937A0000907A0006FC8F
:10198000FCCF70917A00706470937A0000907A00B6
:1019900006FCFCCF809178009091790008959030FA
:1019A00041F00D911C91000F111F9A95E1F71C93C6
:1019B0000E930895903041F00D911C911695079566
:1019C0009A95E1F71C930E930895C89531960020DF
:1019D000089591E005C092E003C094E001C098E052
:1019E000F4DF0D929A95E1F70895E80FF91FF1CF12
:1019F00079910D919981903009F013D0502788E0AA
:101A0000440F551F10F4422753278A95C9F77A953A
:101A100081F789919991803019F08A0105D0A80148
:101A2000089588E0112701C080E1F801F695E79557
:0A1A3000001F111F8A95D1F70895D9
:00000001FF
